:020000020000FC
:0200000009C035
:0200060014C61E
:1000120090C60FEF01BB0FEF02BB0FEF04BB0FEF58
:1000220005BB04E007BB08E308BB0FE50DBF04E016
:100032000EBF00E010E021E031E040E050E060E07F
:1000420070E080E090E000930801009309010093C2
:100052000A0100930B010093010100930201009336
:10006200030100930401009305010093060100932C
:1000720012010093130100931401009315010093E0
:100082001601009317010093190100930D010093CB
:100092000F010093100100931B0100931C010093B8
:1000A2002201009325010093240101E0009318012D
:1000B20000932301009300010093070100930C01B8
:1000C20000930E0100931D0100931E010093210174
:1000D2000093200103E000931F010AE00093110145
:1000E20000E009BF08E002BD03E003BF00E00FBD6E
:1000F2000BE00EBD00E00BBD09E20ABD0BE005BD41
:1001020005E603BD01E809BF02B50830E9F708B703
:100112000660076008BF789400E808B906B301706A
:10012200013061F400E00093250101E809BF00E815
:1001320005BF789488950000F894F0CF08B3047056
:100142000430C9F001E00093250100911E01003046
:1001520031F002B501FDFDCF00E000931E010FEF6B
:1001620002BB05BB00E809BF00EB05BF7894889588
:100172000000F894D3CF01E0009325010FEF02BBFA
:1001820005BB01E809BF00E805BF78948895000027
:10019200F894C4CF213051F0223071F0233091F025
:1001A2002430B9F02530D9F0263001F1042FACD13A
:1001B20002BB01E005BB0895052FA6D102BB02E0F8
:1001C20005BB0895062FA0D1005802BB04E005BB71
:1001D2000895072F99D102BB08E005BB0895082FA7
:1001E20093D1005802BB00E105BB0895092F0030EE
:1001F20011F08AD101C00FEF02BB00E205BB0895E6
:10020200213051F0223069F0233081F02430B1F0F6
:100212002530D9F0263009F107EC02BB01E005BB1D
:10022200089508E802BB02E005BB089500910801A9
:100232006BD1005802BB04E005BB0895009109018F
:1002420063D102BB08E005BB089500910A015CD1AD
:10025200005802BB00E105BB089500910B0100307C
:1002620011F052D101C00FEF02BB00E205BB0895AD
:10027200213051F0223079F02330A9F02430D1F02E
:10028200253001F1263029F1009101013DD102BB57
:1002920001E005BB08950091020136D1005802BB6E
:1002A20002E005BB0895009103012ED102BB04E0D8
:1002B20005BB08950091040127D1005802BB08E054
:1002C20005BB0895009105011FD102BB00E105BBEA
:1002D20008950091060118D1005802BB00E205BB47
:1002E2000895213051F0223081F02330C9F02430BA
:1002F200F9F0253041F1263071F100910C0104D161
:10030200005802BB01E005BB089500910D010030C9
:1003120011F0FAD001C00FEF02BB02E005BB089555
:1003220000910E01F1D0005802BB04E005BB089514
:1003320000910F01003011F0E7D001C00FEF02BBB6
:1003420008E005BB08950091070108D1005802BBDF
:1003520000E105BB08950091070100D112BB00E244
:1003620005BB0895213051F0223079F0233091F00D
:100372002430A9F02530C1F02630E9F000911001B7
:1003820010D102BB01E005BB089507E402BB02E005
:1003920005BB089508E802BB04E005BB08950FEF12
:1003A20002BB08E005BB089500910701D7D002BB4C
:1003B20000E105BB089500910701D0D012BB00E215
:1003C20005BB0895213099F4009112019DD010913E
:1003D2001901113021F41091110110FD0FEF10914C
:1003E200180110FD005802BB01E005BB0895223040
:1003F20079F40091130188D010911901123021F47F
:100402001091110110FD0FEF02BB02E005BB089530
:10041200233099F40091140177D01091190113300F
:1004220021F41091110110FD0FEF10911A0111FF2B
:10043200005802BB04E005BB0895243079F4009112
:10044200150162D010911901143021F4109111019B
:1004520010FD0FEF02BB08E005BB0895253099F4AB
:100462000091160151D010911901153021F410910B
:10047200110110FD0FEF10911A0111FF005802BB7C
:1004820000E105BB0895009117013ED010911901BA
:10049200163021F41091110110FD0FEF02BB00E2A2
:1004A20005BB0895213051F0223079F02330A1F0BC
:1004B2002430B9F02530D1F02630F9F000911F0137
:1004C20023D002BB01E005BB0895009120011CD09E
:1004D20002BB02E005BB08950DEF02BB04E005BBC1
:1004E20008950FEF02BB08E005BB089500912101BA
:1004F20068D002BB00E105BB08950091210161D0E3
:1005020012BB00E205BB08950030A1F00130A1F05A
:100512000230A1F00330A1F00430A1F00530A1F0C7
:100522000630A1F00730A1F00830A1F00930A1F0A7
:100532000FEB089500EC089509EF089504EA089579
:1005420000EB089509E9089502E9089502E8089583
:1005520008EF089500E8089500E90895013061F078
:10056200023069F0033071F0043079F0053081F027
:10057200063089F0073091F003EA1CE8089507E895
:1005820011EC089507E812E9089507E816EC0895BA
:1005920008E81CE8089503EA12E9089506E81BEA50
:1005A2000895003031F0013031F0023031F0033083
:1005B20031F007EF089509EF089502E9089508EF71
:1005C2000895003011F0013019F007EF17EF089588
:1005D20006EA18E8089543954A30E0F040E0539562
:1005E2005630C0F050E063956A3098F060E0739541
:1005F200763078F070E08395DFD08A3010F080E0BA
:100602009395843030F0923020F080E090E003D077
:1006120055D05FD0089500910E01039500930E010D
:100622000A3040F000E000930E0100910F010395A3
:1006320000930F0173D000910F01011748F16ED0A2
:1006420010910E01101720F101E000930E0100E05D
:1006520000930F0100910C01039500930C010A30E5
:1006620040F000E000930C0100910D01039500930E
:100672000D0100910D01013058F000910C01033081
:1006820038F001E000930C0100E000930D0101D06D
:10069200089500911F01039500931F010A3068F02D
:1006A20000E000931F0100912001039500932001B7
:1006B2000A3018F000E0009320010895009107012C
:1006C200039500930701083018F001E00093070139
:1006D200089500911001003001F1013031F0033032
:1006E20021F0009107010630C0F4009108010617BD
:1006F200A1F400910901071781F400910A0108177A
:1007020061F400910B01091741F4C29A00911001A2
:10071200013019F400E000931001089500910C01DA
:1007220010910D01103019F00395039503950130D6
:1007320081F0023089F00330C1F00430C9F0053095
:10074200D1F00630D9F00730E1F00830E9F0093095
:10075200F1F013E002E008951DD0103019F412E018
:1007620009E0089513E000E0089513E002E008951F
:1007720013E001E0089513E002E0089513E001E0C0
:10078200089513E002E0089513E002E0089513E0F3
:1007920001E008951091200100911F0111701130A4
:1007A20011F40395039511E0003029F0043019F09B
:1007B200083009F010E0089500912101003071F134
:1007C20000910F01003051F1013041F1033021F06D
:1007D20000910E01053010F1009107010730F1F48C
:1007E20000910C01033029F000910C01003041F01E
:1007F20015C0823099F4903089F483E090E0089536
:1008020000912201013051F0833041F4903031F4F3
:1008120082E090E001E000932201089500E000935D
:1008220022010895009112010A95009312010F3FCF
:1008320099F509E000931201009113010A950093C2
:1008420013010F3F49F505E00093130100911401D4
:100852000A95009314010F3FF9F409E00093140183
:10086200009115010A95009315010F3FA9F405E0C7
:1008720000931501009116010A95009316010F3F8E
:1008820059F409E000931601009117010A950093AB
:1008920017010F3F09F401D0089500E000931701FA
:1008A20000931601009315010093140100931301A4
:1008B2000093120101E000931801C29A0895009179
:1008C2001C01003019F00A9500931C0110911B01C4
:1008D20006B3087300931B01101781F010911C01DD
:1008E200103061F403FF05C004FF05C005FF05C019
:1008F20005C0CCD003C02DD001C090D115E003FFBC
:1009020010931C0104FF10931C0105FF10931C019E
:10091200083329F0109126011395109326011091A6
:100922001C01103019F410E01093260110912601D9
:10093200143671F41CE51093260103FF05C004FF71
:1009420005C005FF05C004C0A1D002C002D000C08E
:1009520008950091250100FD0895313071F0323083
:1009620069F0333061F0343059F0353051F03630BF
:1009720049F0373041F0383039F007C013C030C089
:1009820044C063C064C06BC078C083958A3010F0E5
:1009920080E09395843020F0923010F080E090E077
:1009A20098DE089500910A01039500930A010A3026
:1009B20040F000E000930A0100910B0103950093BF
:1009C2000B0100910B01023048F000910A01043042
:1009D20028F000E000930A0100930B017ADE0895EB
:1009E20000910001023069F000E0009301010093E0
:1009F2000201009303010093040100930501009397
:100A0200060101E000930001089500910E01039593
:100A120000930E010A3040F000E000930E010091B5
:100A22000F01039500930F0179DE00910F01011769
:100A320058F074DE10910E01101730F001E00093AF
:100A42000E0100E000930F01089538DE0895009131
:100A52002301053019F003950093230108950091B5
:100A6200180101E00093180100911901003009F406
:100A720007E00A9500931901089500912101039559
:100A8200023008F000E00093210108950091250151
:100A920000FD0895313071F0323069F0333061F089
:100AA200343059F0353051F0363049F0373041F0BA
:100AB200383039F007C015C02AC031C04EC056C008
:100AC2005DC0AAC063956A3028F060E07395763005
:100AD20008F070E040E050E00AE000931101F9DD17
:100AE2000895009108010395009308010A3068F007
:100AF20000E00093080100910901039500930901A8
:100B0200063018F000E000930901E3DD089500913A
:100B120000010A9509F402E0009300010895009192
:100B22000C01039500930C010A3040F000E00093A1
:100B32000C0100910D01039500930D0100910D012F
:100B4200013050F000910C01033030F001E00093CD
:100B52000C0100E000930D0108950091100103952E
:100B6200043008F000E00093100108950091230181
:100B7200003019F00A95009323010895009119019C
:100B8200003061F0013091F00230C9F0033001F120
:100B9200043039F1053071F10630A9F100911801E4
:100BA2000A9509F402E000931801089500911201D8
:100BB20003950A3008F000E00093120108950091B5
:100BC20013010395063008F000E000931301089525
:100BD2000091140103950A3008F000E0009314011B
:100BE2000895009115010395063008F000E0009386
:100BF200150108950091160103950A3008F000E0EE
:100C02000093160108950091170103950A3008F028
:100C120000E00093170108953CDD089508B30470C5
:100C2200043019F03A9509F438E0C2980895009119
:100C32001D010A9509F40AE000931D010A3019F01A
:100C4200063039F00BC016E613BD01E000931E0119
:100C520005C015E613BD01E000931E0100911101CC
:100C62000A9579F4B8DC09E2041B041B0ABD00E012
:100C72000DBD00E00CBD00911801023009F4D2DD77
:100C82000AE000931101009100010230E1F50091A8
:100C920001010395009301010A30A8F100E00093DD
:100CA2000101009102010395009302010A3058F1FB
:100CB20000E00093020100910301039500930301F8
:100CC200063008F100E0009303010091040103954E
:100CD200009304010A30B8F000E00093040100918F
:100CE2000501039500930501063068F000E00093CA
:100CF2000501009106010395009306010A3018F0E0
:100D020000E00093060100911A010A9509F405E03A
:100D120000931A0110E008B30470043039F4009112
:100D22001A0100FD03C010E4B99A01C0B9981FBDB1
:100D320018950091240110912301103051F01130C7
:100D420051F0123051F0133051F0143051F015308F
:100D520051F018E909C01CEC07C016EE05C013EFEC
:100D620003C019EF01C01CEF013011F0003089F00F
:100D72000FEF011B17E6101B0FEF011B02BF00E074
:100D82000093240100912501013081F000E005BBB0
:100D9200189512BF01E0009324012A9511F426E070
:100DA2008EDD00912501013009F001D0189500E097
:100DB20005BB313071F0323071F0333071F03430C4
:100DC20071F0353071F0363071F0373089F03830EB
:100DD20089F0E0D911C014DA0FC04ADA0DC081DA05
:100DE2000BC0C0DA09C040FFD5D940FD7ADA04C091
:0A0DF200E9DA02C057DB00C00895E3
:00000001FF
